S31508000000F82B002069020008611E0008171A00086C
S315080000105D1E000809070008654B0008000000007F
S3150800002000000000000000000000000085460008EF
S315080000301507000800000000750600089102000870
S31508000040930200089302000893020008930200082E
S31508000050930200089302000893020008930200081E
S31508000060930200089302000893020008930200080E
S3150800007093020008930200089302000893020008FE
S3150800008093020008930200089302000893020008EE
S3150800009093020008930200089302000893020008DE
S315080000A093020008930200089302000893020008CE
S315080000B093020008930200089302000893020008BE
S315080000C093020008930200089302000893020008AE
S315080000D09302000893020008994A00089302000850
S315080000E0930200089302000893020008930200088E
S315080000F0930200089302000893020008930200087E
S31508000100930200089302000893020008930200086D
S31508000110930200089302000893020008930200085D
S31508000120930200089302000893020008930200084D
S31508000130930200089302000893020008930200083D
S31508000140930200089302000893020008930200082D
S31508000150930200089302000893020008930200081D
S31508000160930200089302000893020008930200080D
S31508000170930200089302000893020008000000009A
S31508000180930200089302000800F002F800F05CF8F9
S315080001900AA090E8000C82448344AAF10107DA45D4
S315080001A001D100F051F8AFF2090EBAE80F0013F0CA
S315080001B0010F18BFFB1A43F0010318474454000007
S315080001C0645400000A444FF0000C10F8013B13F089
S315080001D0070408BF10F8014B1D1108BF10F8015B92
S315080001E0641E05D010F8016B641E01F8016BF9D185
S315080001F013F0080F1EBF10F8014BAD1C0C1B09D1DC
S315080002006D1E58BF01F801CBFAD505E014F8016B4D
S3150800021001F8016B6D1EF9D59142D6D370470000DF
S315080002200023002400250026103A28BF78C1FBD8F1
S31508000230520728BF30C148BF0B6070471FB505F08D
S31508000240CDF81FBD10B510BD00F09EF91146FFF799
S31508000250F5FF04F0A5FF00F0BCF903B4FFF7F2FFC1
S3150800026003BC04F059FE0000DFF83400016841F4CD
S3150800027070010160BFF34F8F0A4880470A4800475C
S31508000280FEE7FEE7FEE7FEE7FEE7FEE7FEE7FEE738
S31508000290FEE7FEE705480649044A064B7047000094
S315080002A088ED00E08946000889010008F827002043
S315080002B0F82B0020F827002072B6704762B6704700
S315080002C072B602B4EFF3118180F31188BFF34F8F32
S315080002D0BFF36F8F084602BC62B6704772B680F3EA
S315080002E01188BFF34F8FBFF36F8F62B6704730BF69
S315080002F0704720BF7047B0FA80F0704790FAA0F0B8
S31508000300B0FA80F0704790FAA0F07047704753EA49
S31508000310020C00F069802DE9F04B4FF00006002B27
S315080003201FBFB3FA83F503FA05F424FA05F65E400F
S3150800033012BF1643B2FA82F502FA05F4C5F1200592
S315080003401EBF22FA05FC44EA0C04203556EA044C82
S315080003504FEA144418BF641C4FF000084FF0000918
S31508000360904271EB030C39D3002919BFB1FA81F712
S3150800037001FA07F6B0FA80F700FA07F6C7F1200780
S315080003801EBF20FA07FC46EA0C062037B6FBF4FC2B
S31508000390A7EB0507103F07F01F0BCBF120060CFA59
S315080003A00BFB2CFA06F644BFB3460026202FA4BF43
S315080003B05E464FF0000B5BEA060C08BF4FF0010BD8
S315080003C019EB0B09ABFB027C48EB0608C01B06FBC6
S315080003D002CC0BFB03CC71EB0C01C1E70B460246C2
S315080003E041464846BDE8F08B13B54FF000004FF084
S315080003F00001AFF30080BDE81C40704740EA0103E6
S31508000400024630B59B0710D14FF0013400E008C210
S3150800041008C91D1B9D4315EAC41FF8D013F0FF0138
S3150800042002F8011B0DD01B0AF8E711F8013B002B57
S3150800043002F8013B05D011F8013B002B02F8013BFD
S31508000440F3D130BD032A40F2308010F0030C00F0DF
S31508000450158011F8013BBCF1020F624498BF11F8F0
S3150800046001CB00F8013B38BF11F8013BA2F10402A9
S3150800047098BF00F801CB38BF00F8013B11F0030321
S3150800048000F05080083AC0F0088051F8043B083A5A
S3150800049051F804CBA0E80810F5E7121D5CBF51F827
S315080004A0043B40F8043BAFF30080D20724BF11F8A1
S315080004B0013B11F801CB48BF11F8012B24BF00F806
S315080004C0013B00F801CB48BF00F8012B70474FF0FD
S315080004D0000200B5134694469646203922BFA0E886
S315080004E00C50A0E80C50B1F12001BFF4F7AF090792
S315080004F028BFA0E80C5048BF0CC05DF804EB890083
S3150800050028BF40F8042B08BF704748BF20F8022BC5
S3150800051011F0804F18BF00F8012B704770477047DD
S315080005207047704710B5203AC0F00B80B1E81850F4
S31508000530203AA0E81850B1E81850A0E81850BFF4BF
S31508000540F5AF5FEA027C24BFB1E81850A0E818505E
S3150800055044BF18C918C0BDE810405FEA827C24BFB2
S3150800056051F8043B40F8043B08BF7047D20728BF40
S3150800057031F8023B48BF11F8012B28BF20F8023B8F
S3150800058048BF00F8012B7047754600F02BF8AE46B9
S3150800059005006946534620F00700854618B020B581
S315080005A0FFF778FEBDE820404FF000064FF0000741
S315080005B04FF000084FF0000B21F00701AC46ACE8FD
S315080005C0C009ACE8C009ACE8C009ACE8C0098D466A
S315080005D0704710B50446AFF300802046BDE81040CA
S315080005E0FFF73BBE004870479427002072B64EF6C8
S315080005F02250CEF2000040F2FF01C0F20001017065
S31508000600002080F3098841F28800C2F200000168E0
S3150800061081F3088802F0C0FA41F2B600C2F200007F
S3150800062041F2B701C2F200010A78027041F23010B5
S31508000630C2F2000041F23411C2F200010A680260F7
S31508000640106880F30988EFF3148040F0020020F068
S31508000650040080F31488BFF36F8FBDE8F04F0FBC1A
S31508000660BDE8005006BC62B6084726484FF08051E0
S315080006700160704772B641F28C02C2F2000211683C
S3150800068081F31188BFF34F8FBFF36F8F62B6EFF315
S3150800069009801EF0100F08BF20ED108A20E9F04FE0
S315080006A041F23015C2F2000529680860744602F066
S315080006B073FA41F2B600C2F2000041F2B701C2F283
S315080006C000010A78027041F23411C2F200010A6888
S315080006D02A6044F0040E1068B0E8F04F1EF0100FC0
S315080006E008BFB0EC108A80F3098840F20002C0F215
S315080006F0000272B682F31188BFF34F8FBFF36F8F74
S3150800070062B6704704ED00E000BFFEE700BFFEE7F3
S315080007100020704770470000F0B504460A46216875
S3150800072094F82050012D01D0022D7ED1424901F5C1
S315080007300071086840F001000860086820F47C50E1
S3150800074008600868566A40EA06200860107D00F0CE
S315080007501F06012000FA06F3C8699843C861A1F587
S315080007600071D069C8B9D1F80C029843C1F80C02D7
S31508000770908880B2968940EA064601F51070576956
S3150800078040F83760108880B2168940EA064601F5B7
S315080007901070576900EBC7004660D069012819D167
S315080007A0D1F80C021843C1F80C02908880B216885A
S315080007B040EA064601F51070576940F83760908997
S315080007C080B2168940EA064601F51070576900EBB3
S315080007D0C7004660906928B9D1F804029843C1F861
S315080007E0040204E0D1F804021843C1F804021069AF
S315080007F028B9D1F814029843C1F8140204E0D1F8D4
S3150800080014021843C1F81402106A012804D1D1F859
S315080008101C021843C1F81C02D1F8000220F001009E
S31508000820C1F800020020F0BDFFE7606A40F48020AE
S3150800083060620120F7E700000064004070B50446D6
S315080008400CB9012070BD94F8200010B9204600F0BC
S31508000850AFF82068006820F002002168086000F000
S31508000860A7FA05460DE000F0A3FA401B0A2808D9A6
S31508000870606A40F400306062052084F82000012098
S31508000880E0E72068406800F002000028EBD1206805
S31508000890006840F001002168086000F089FA054602
S315080008A00DE000F085FA401B0A2808D9606A40F472
S315080008B000306062052084F820000120C2E7206825
S315080008C0406800F001000028EBD0207E012806D100
S315080008D02068006840F080002168086005E020680C
S315080008E0006820F0800021680860607E012806D133
S315080008F02068006840F040002168086005E020682C
S31508000900006820F0400021680860A07E012806D112
S315080009102068006840F020002168086005E020682B
S31508000920006820F0200021680860E07E012806D1D2
S315080009302068006820F010002168086005E020683B
S31508000940006840F0100021680860207F012806D161
S315080009502068006840F008002168086005E0206803
S31508000960006820F0080021680860607F012806D129
S315080009702068006840F004002168086005E02068E7
S31508000980006820F0040021680860D4E902010843E1
S3150800099021690843616908436168491E084321685B
S315080009A0C86100206062012084F82000002049E721
S315080009B010B586B004462849206888424AD100BF47
S315080009C000BF002000902548006840F00100234938
S315080009D008600846006800F00100009000BF00BFEC
S315080009E000BF00BF00BF002000900846006840F026
S315080009F0010008600846006800F00100009000BF8A
S31508000A0000BF00BF00BF00200090144810300068E7
S31508000A1040F000701149103108600846006800F07F
S31508000A200070009000BF00BF881401900220029059
S31508000A3001200390022004900920059001A9084886
S31508000A4000F0A8F84FF40060019001A9044800F0EE
S31508000A50A1F800BF06B010BD00640040303802405F
S31508000A600000024070B5044694F82000012822D1FF
S31508000A70022084F820002068006820F00100216820
S31508000A80086000F095F905460DE000F091F9401B65
S31508000A900A2808D9606A40F400306062052084F8A4
S31508000AA02000012070BD2068406800F00100002881
S31508000AB0EBD16062F6E7606A40F4002060620120CC
S31508000AC0F0E770B50446A56D00F072F9064694F88D
S31508000AD03500022808D08020606500BF002084F811
S31508000AE0340000BF012070BD2068006820F01600A1
S31508000AF0216808602068406920F080002168486104
S31508000B00206C08B9A06C28B12068006820F008009D
S31508000B10216808602068006820F0010021680860E4
S31508000B200FE000F045F9801B05280AD920206065EA
S31508000B3000BF002084F8340000BF032084F8350085
S31508000B40D1E72068006800F001000028E9D194F890
S31508000B505C103F208840A86000BF002084F834005D
S31508000B6000BF012084F835000020BCE7014691F853
S31508000B703500022803D080204865012070470520EB
S31508000B8081F835000868006820F001000A681060DE
S31508000B900020F3E7F8B502460B460025002400209E
S31508000BA00021DEE0012606FA01F51E6806EA0504BC
S31508000BB0AC4275D11E7906F00306012E04D01E79C3
S31508000BC006F00306022E13D190684F000326BE4096
S31508000BD0B0434F00DE68BE4030439060506801263F
S31508000BE08E40B0431E79C6F300168E4030435060DF
S31508000BF01E7906F00306032E09D0D0684F00032697
S31508000C00BE40B0434F009E68BE403043D0601E7958
S31508000C1006F00306022E13D1CF0802F1200656F875
S31508000C2027004E07F70E0F26BE40B0434F07FF0EAC
S31508000C301E69BE403043CF0802F1200646F8270059
S31508000C4010684F000326BE40B0431E7906F003061F
S31508000C504F00BE40304310605E6806F08056B6F11D
S31508000C60805F7DD100BF00260096404E366846F468
S31508000C7080463E4F3E603E46366806F480460096FD
S31508000C8000BF00BF3A4E8F0856F827008E07370F69
S31508000C900F26BE40B043374EB24202D1002624E0AA
S31508000CA05EE0354EB24201D101261EE0334EB24215
S31508000CB001D1022619E0324EB24201D1032614E0D0
S31508000CC0304EB24201D104260FE02F4EB24201D176
S31508000CD005260AE02D4EB24201D1062605E02C4E25
S31508000CE0B24201D1072600E008268F073F0FBE4013
S31508000CF030431F4E8F0846F82700264E3068A0431B
S31508000D005E6806F48036B6F5803F00D12043214E52
S31508000D103060361D3068A0435E6806F40036B6F5C6
S31508000D20003F00D120431B4E361D3060361D30680B
S31508000D30A0435E6806F48016B6F5801F00D12043EE
S31508000D40144E08363060361D3068A0435E6806F4D7
S31508000D500016B6F5001F00D120430E4E0C36306043
S31508000D60491C1029FFF41EAFF8BD000044380240A4
S31508000D700838014000000240000402400008024012
S31508000D80000C024000100240001402400018024005
S31508000D90001C0240003C01400AB1816101E00B04DD
S31508000DA08361704701480068000C7047002004E022
S31508000DB001480068704700007810002010B50A48FE
S31508000DC0006840F40070084908600846006840F466
S31508000DD080600860032000F07FF80F2000F006F816
S31508000DE000F02AF8002010BD003C024070B5044609
S31508000DF00E4800784FF47A71B1FBF0F00C49096897
S31508000E00B1FBF0F5284600F01DFC08B1012070BDC5
S31508000E10102C07D200222146501E00F01EF8054865
S31508000E20046001E00120F2E70020F0E780100020CE
S31508000E30841000207C1000207047014608460028D0
S31508000E4009DB00F01F0301229A4043099B0003F1C6
S31508000E50E023C3F8002100BF70472DE9F05F804604
S31508000E600D461646002704F03BF8074639462A463B
S31508000E70334601F00700C0F1070ABAF1040F02D998
S31508000E804FF0040A01E0C0F1070AD14600F1040A4E
S31508000E90BAF1070F02D24FF0000A01E0A0F1030AE7
S31508000EA0D4464FF0010A0AFA09FAAAF1010A0AEA2F
S31508000EB0020A0AFA0CFA4FF0010B0BFA0CFBABF11B
S31508000EC0010B0BEA030B4AEA0B042146404604F0E1
S31508000ED00FF8BDE8F09F000000BF00F00702064BC0
S31508000EE019684FF6FF031940044B0B4343EA0221E6
S31508000EF0014B196000BF70470CED00E00000FA05D1
S31508000F0070B504460D460CB9012070BD58480068F6
S31508000F1000F00700A84209D255490D700846006836
S31508000F2000F00700A84201D00120EEE7207800F083
S31508000F30020002281DD1207800F00400042805D1FB
S31508000F404C48006840F4E0504A490860207800F0B0
S31508000F500800082805D14748006840F4604045491C
S31508000F6008604448006820F0F000A1680843414939
S31508000F700860207800F00100A8B36068012807D14E
S31508000F803C4808380068C0F34040B8B90120BCE7BF
S31508000F906068022802D06068032807D135480838F7
S31508000FA00068C0F3406048B90120AEE73148083808
S31508000FB00068C0F3400008B90120A6E72D4800687C
S31508000FC020F00300616808432A490860FFF7F0FE2D
S31508000FD0064609E0FFF7ECFE801B41F2883188429D
S31508000FE002D9032091E707E02248006800F00C00C8
S31508000FF06168B0EB810FEDD11D48006800F007006D
S31508001000A84209D91A490D700846006800F0070079
S31508001010A84201D0012078E7207800F004000428CF
S3150800102007D11448006820F4E050E16808431149E4
S315080010300860207800F00800082808D10D480068E4
S3150800104020F46040216940EAC1000A49086000F0BE
S315080010503FF808490968C1F30311074A515CC840BB
S315080010600649086006480068FFF7C0FE00204CE7FE
S31508001070003C0240083802400C5400088410002046
S315080010807C1000200148006870470000841000208A
S3150800109000B5FFF7F7FF04490968C1F38221034A3F
S315080010A0515CC84000BD0000083802401C540008C6
S315080010B000B5FFF7E7FF04490968C1F34231034A5F
S315080010C0515CC84000BD0000083802401C540008A6
S315080010D02DE9F047002400250026A146254800688A
S315080010E000F00C0020B1042805D008283AD105E004
S315080010F0DFF8849039E0DFF8849036E01D48001F59
S31508001100006800F03F041B48001F006800F48000D8
S3150800111078B11A481749091F0968C1F38811A0FB55
S3150800112001700146224600233846FFF7F0F80546C7
S315080011300EE011480F49091F0968C1F38811A0FB81
S3150800114001700146224600233846FFF7E0F80546B7
S315080011500848001F0068C0F30140401C4600B5FB64
S31508001160F6F902E0DFF8109000BF00BF4846BDE878
S31508001170F0870000083802400024F40000127A00C4
S31508001180F8B504460CB90120F8BD207800F0010036
S31508001190002874D0F948006800F00C0004280DD027
S315080011A0F648006800F00C00082813D1F348001F21
S315080011B0006800F48000B0F5800F0BD1EF480838BE
S315080011C00068C0F34040002859D06068002856D10E
S315080011D00120D9E700BF6068B0F5803F08D1E7482D
S315080011E00838006840F48030E449083908601EE091
S315080011F06068B0F5A02F0DD1E0480838006840F4C3
S315080012008020DE49083908600846006840F48030C6
S3150800121008600CE0D9480838006820F48030D749BF
S31508001220083908600846006820F48020086000BF76
S31508001230606890B1FFF7BCFD054606E0FFF7B8FD0C
S31508001240401B642801D903209EE7CC48083800686B
S31508001250C0F340400028F1D011E0FFF7A9FD05468C
S3150800126006E0FFF7A5FD401B642801D903208BE79C
S31508001270C24808380068C0F340400028F1D12078F9
S3150800128000F0020002285FD1BC48006800F00C009C
S3150800129058B1BA48006800F00C0008281CD1B748B5
S315080012A0001F006800F48000B0B9B4480838006828
S315080012B0C0F3400020B1E068012801D0012063E7AF
S315080012C0AE480838006820F0F800216940EAC100F5
S315080012D0AA490839086037E0E06800B30120A84940
S315080012E00860FFF765FD054606E0FFF761FD401B50
S315080012F0022801D9032047E7A04808380068C0F348
S3150800130040000028F1D09D480838006820F0F80011
S31508001310216940EAC10099490839086014E00020AB
S3150800132097490860FFF744FD054606E0FFF740FDCC
S31508001330401B022801D9032026E790480838006890
S31508001340C0F340000028F1D1207800F008000828F2
S315080013502CD16069A8B101208A490860FFF728FDE9
S31508001360054606E0FFF724FD401B022801D90320A5
S315080013700AE782486C300068C0F340000028F1D0C4
S3150800138014E000207F490860FFF712FD054606E0D5
S31508001390FFF70EFD401B022801D90320F4E6774823
S315080013A06C300068C0F340000028F1D1207800F0C6
S315080013B00400042870D1002770483830006800F00F
S315080013C0805090B900BF002000906C483830006803
S315080013D040F080506949383108600846006800F0D6
S315080013E08050009000BF00BF01276748006800F4DE
S315080013F08070B0B96448006840F48070624908603B
S31508001400FFF7D6FC054606E0FFF7D2FC401B02288C
S3150800141001D90320B8E65C48006800F4807000280B
S31508001420F2D000BFA068012808D154486830006887
S3150800143040F001005149683108601DE0A0680528A0
S315080014400DD14E486830006840F004004B496831B9
S3150800145008600846006840F0010008600CE047484C
S315080014606830006820F00100444968310860084681
S31508001470006820F00400086000BFA068A8B1FFF764
S3150800148097FC054609E0FFF793FC401B41F28831BB
S31508001490884202D9032077E626E038486830006893
S315080014A0C0F340000028EED013E0FFF781FC0546A4
S315080014B008E0FFF77DFC401B41F28831884201D9DC
S315080014C0032061E62D4868300068C0F34000002814
S315080014D0EFD1012F07D129483830006820F0805015
S315080014E026493831086000BFA069002845D023483E
S315080014F0006800F00C0008285DD0A069022845D1D4
S3150800150000201F490866FFF753FC054606E0FFF76B
S315080015104FFC401B022801D9032035E61748083836
S315080015200068C0F340600028F1D1D4E907010843F8
S31508001530616A40EA81110122A06AC2EB500041EAC1
S3150800154000412C20005D41EA00600C49091F086033
S3150800155001200B490866FFF72BFC054606E0FFF756
S3150800156027FC401B022801D903200DE6034808384A
S315080015700068C0F340600028F1D049E0083802400E
S3150800158000004742800E4742007000400020214973
S315080015900866FFF70DFC054606E0FFF709FC401B49
S315080015A0022801D90320EFE51B480068C0F3406014
S315080015B00028F2D12CE0A069012800D1E4E51648FC
S315080015C0001D0668A069012820D006F48001E0699C
S315080015D081421BD106F03F01206A814216D147F6A7
S315080015E0C0703040616AB0EB811F0FD106F44031FC
S315080015F00122A06AC2EB5000B1EB004F06D106F0FB
S3150800160070612C20005DB1EB006F01D00120BBE5B5
S315080016100020B9E50000474200380240042808D1F6
S315080016204FF0E021096941F004014FF0E022116111
S3150800163007E04FF0E021096921F004014FF0E022AC
S315080016401161704770B504462546681EB0F1807F63
S3150800165001D301200FE0681E4FF0E02148610F21F9
S315080016604FF0FF3003F044FC00204FF0E021886182
S3150800167007200861002070BD7047704701460022A8
S31508001680002391F83D2091F83E3042EA0300704766
S315080016902DE9F84F0446206805682068C668206862
S315080016A047694FF00009CA4605F00F09B9F1000F5E
S315080016B00AD105F0200038B106F0200020B12046F6
S315080016C003F021F8BDE8F88FB9F1000F72D007F0E2
S315080016D0010018B906F4907000286BD005F00100D7
S315080016E030B106F4807018B1206C40F00100206417
S315080016F005F0040030B107F0010018B1206C40F085
S315080017000200206405F0020030B107F0010018B1AC
S31508001710206C40F00400206405F0080048B106F08B
S31508001720200010B907F0010018B1206C40F008003D
S315080017302064206C70B305F0200028B106F0200064
S3150800174010B1204602F0DFFF20684069C0F3801A16
S31508001750206C00F0080010B9BAF1000F23D020461B
S3150800176002F0A6FF2068406900F04000402816D124
S315080017702068406920F0400021684861A06B50B19C
S315080017805648A16B0865A06BFFF7F0F910B1A06B7E
S31508001790016D88470CE02046FFF76FFF08E02046FA
S315080017A0FFF76BFF04E02046FFF767FF0020206481
S315080017B088E7FFE7206B012879D105F0100000289B
S315080017C075D006F01000002871D000BF00200090E8
S315080017D020680068009020684068009000BF00BF3D
S315080017E02068406900F04000402839D1A06B0068A5
S315080017F040681FFA80F8B8F1000F30D0A08D404538
S315080018002DDDA4F82E80A06BC069B0F5807F1FD0AF
S315080018102068C06820F480702168C8602068406924
S3150800182020F00100216848612068406920F04000E6
S3150800183021684861202084F83E0000202063206843
S31508001840C06820F010002168C860A06BFFF739F95E
S31508001850A08DE28D801A81B22046FFF70DFF31E791
S31508001860A08DE18D401A1FFA80F8E08DE8B1B8F135
S31508001870000F1AD02068C06820F490702168C860EC
S315080018802068406920F0010021684861202084F81A
S315080018903E00002020632068C06820F01000216800
S315080018A0C86041462046FFF7E7FE0BE7FFE705F06D
S315080018B0800030B106F0800018B1204603F0BBF86E
S315080018C000E705F0400030B106F0400018B12046A8
S315080018D002F009FFF6E600BFF4E600009D460008A0
S315080018E010B504460CB9012010BDA06900B100E08E
S315080018F000BF94F83D0028B9002084F83C00204633
S3150800190000F027F8242084F83D002068C06820F4F9
S3150800191000502168C860204602F054FF206800691C
S3150800192020F49040216808612068406920F02A0068
S31508001930216848612068C06840F400502168C86082
S3150800194000202064202084F83D0084F83E00002012
S31508001950CAE7704770B504460D46164694F83E0029
S31508001960202816D105B10EB9012070BD00BF94F824
S315080019703C00012801D10220F7E7012084F83C0049
S3150800198000BF0020206332462946204603F030F87F
S31508001990EBE70220E9E700001B49098801F400414A
S315080019A089BB1949098801F4804171B11749097839
S315080019B00A2903D00021144A118024E01249098813
S315080019C041F40041104A11801DE0104909780D299B
S315080019D006D10D49098841F480410B4A118012E06D
S315080019E00A490978084A1288C2F30D02084B995425
S315080019F005490988491C044A118011460988C729DE
S31508001A0001DD002111807047680E00206A0E002053
S31508001A1038110020704700BFFEE7000010B586B0F9
S31508001A2000BF002000905948006840F0010057495F
S31508001A3008600846006800F00100009000BF00BF7B
S31508001A4000BF002000900846006840F002000860C9
S31508001A500846006800F00200009000BF00BF00BF03
S31508001A60002000900846006840F004000860084618
S31508001A70006800F00400009000BF00BF00BF00200F
S31508001A8000900846006840F0800008600846006834
S31508001A9000F08000009000BF00BF00BF002000904B
S31508001AA00846006840F0080008600846006800F02C
S31508001AB00800009000BF00BF00BF00200090084645
S31508001AC0006840F0100008600846006800F0100042
S31508001AD0009000BF00BF00BF0020009008460068C5
S31508001AE040F0200008600846006800F020000090DA
S31508001AF000BF00BF00BF002000900846006840F401
S31508001B00807008600846006800F48070009000BF86
S31508001B1000BF00BF002000900846006840F0400063
S31508001B2008600846006800F04000009000BF00BF4B
S31508001B30002427E004EB4400154901EBC000808827
S31508001B40019004EB440001EBC0008068029004EBAE
S31508001B50440001EBC000C068039004EB440001EBAD
S31508001B60C0000069049004EB440001EBC000406922
S31508001B70059004EB4401064A52F8310001A9FFF723
S31508001B8009F8641C102CD5D306B010BD30380240B5
S31508001B90F40E002030B587B00546142102A8FEF7DA
S31508001BA096FC00BF00200190A148006840F0100094
S31508001BB09F4908600846006800F01000019000BFC1
S31508001BC000BF00BF00200190081F006840F40030E5
S31508001BD0091F08600846006800F40030019000BF3D
S31508001BE000BF00BF002001900846006840F480202E
S31508001BF008600846006800F48020019000BF00BF16
S31508001C0000BF002001900846006840F400200860E4
S31508001C100846006800F40020019000BF00BF00BF1E
S31508001C200020019082481438006840F0010080497D
S31508001C30143908600846006800F00100019000BFEA
S31508001C4000BF00BF002001900846006840F0080069
S31508001C5008600846006800F00800019000BF00BF51
S31508001C600024CEE004EB440000EBC400714901EB0C
S31508001C70800000890290022003900020049003202F
S31508001C8005900720069004EB440101EBC401694A5C
S31508001C9002EB8101486802A9FEF77CFF04EB4400C9
S31508001CA000EBC400634901EB8000008A029007201C
S31508001CB0069004EB440101EBC4015E4A02EB810184
S31508001CC0C86802A9FEF766FF04EB440000EBC400EF
S31508001CD0584951F8200004EB0411574A42F82100EC
S31508001CE004EB0410114601EB8000456004EB440048
S31508001CF000EBC4004F4901EB8000416904EB041076
S31508001D0002EB8000816004EB440000EBC400494903
S31508001D1001EB8000816904EB041002EB8000C160CE
S31508001D2004EB440000EBC400424901EB8000C169A2
S31508001D3004EB041002EB8000016104EB440000EBA5
S31508001D40C4003C4901EB8000016A04EB041002EB75
S31508001D508000416104EB440000EBC400354901EB07
S31508001D608000416A04EB041002EB8000816104EBF9
S31508001D70440000EBC4002F4901EB8000816A04EBA4
S31508001D80041002EB8000C16104EB041102EB810030
S31508001D90FFF7A6FD04EB440000EBC400254951F803
S31508001DA020002649884207D1012203212520FFF772
S31508001DB054F82520FFF741F804EB440000EBC40073
S31508001DC01C4951F820001E49884207D102220321E6
S31508001DD02720FFF742F82720FFF72FF804EB4400E7
S31508001DE000EBC400134951F820001649884207D170
S31508001DF0032211463420FFF730F83420FFF71DF888
S31508001E00641C032CFFF42EAF0F4802880F491048B4
S31508001E10FFF7A0FD0C4802880C490E48FFF79AFD0B
S31508001E200948028809490C48FFF794FD07B030BDF8
S31508001E3044380240700E0020CC12002000100140E9
S31508001E4000480040004C00406C0E00206A0E00203E
S31508001E5000120020441200208812002000BFFEE76E
S31508001E607047704770B5044600F09EF8002039495F
S31508001E70087039490870394908703949086039497C
S31508001E80086039490870394908703949087039486D
S31508001E9000680A21B0FBF1F0374908603748056841
S31508001EA045B13748066803E0761E002028602D1DD8
S31508001EB0002EF9D1324801683048006801F0B0FEBA
S31508001EC001F094FA01F0B6FA00202E4908602E496E
S31508001ED00880204601F07CF8208800B170BD2046B5
S31508001EE001F082F8208800B1F8E700202749086049
S31508001EF02749088027490860274908802749086034
S31508001F0027490880204601F005FE208800B1E5E74C
S31508001F10204601F025F8208800B1DFE7204601F0C9
S31508001F208BFE208800B1D9E7204601F0BFFC208847
S31508001F3000B1D3E7204602F041F8208800B1CDE78A
S31508001F4000F0D6FEFFF78DFF01201649087000BF86
S31508001F50C4E700009410002095100020C21000204D
S31508001F603011002034110020B6100020B7100020D0
S31508001F70C810002078540008C410002044540008F3
S31508001F8048540008A0100020A4100020B01000201B
S31508001F90B4100020BC100020C0100020CC10002077
S31508001FA0D0100020961000200C4909680C4A1268C7
S31508001FB001EB82010B4A11601146096821F00701FD
S31508001FC011600949086800F04041B1F1404F01D05D
S31508001FD000BFFEE74021054A1160704744540008D7
S31508001FE0485400088810002034EF00E08C100020C8
S31508001FF070B5002538480078012800D070BD00BFAC
S315080020004020FEF75DF9054600BF3448007828B938
S3150800201000BF2846FEF762F900BFEFE72F480078B1
S31508002020401E2E4908700846007828B100BF284689
S31508002030FEF754F900BFE1E72948007828B100BF48
S315080020402846FEF74BF900BFD8E726480168264818
S31508002050006801F0D1FD0446012C02D0002000F0F2
S31508002060ABF901F0B9F9214908700846007800EB88
S3150800207040001F4951F820001E49086008460068BC
S315080020801D49096888420FD1002000F069FD044601
S31508002090012C03D01848006800F08EF900BF2846C6
S315080020A0FEF71CF900BFA9E712480068D0F89400AB
S315080020B0401C10490968C1F8940010480068401C83
S315080020C00E490860FEF7D1FA00BF2846FEF706F962
S315080020D000BF00BF92E70000951000209410002072
S315080020E0C21000204854000844540008B7100020C5
S315080020F0382400203411002030110020F010002070
S315080021002DE9F04104460E46154600272148007879
S3150800211020B142F6E1602880BDE8F0811CB945F699
S31508002120C3502880F8E700BF00BF4020FEF7C8F874
S31508002130074600BF00BF1849206888420AD100BF79
S3150800214000BF3846FEF7CAF800BF00BF45F6C150C3
S315080021502880E1E7104820606660002020626062FF
S3150800216084F82800E06204F1080001F080F82046AF
S3150800217000F0A0FF09480088401C0849088000BFF5
S3150800218000BF3846FEF7AAF800BF00BF0020288027
S3150800219000BFC1E7941000204D555458B4100020D4
S315080021A02DE9F0470646894617461C46089D4FF016
S315080021B0000A7C48007820B146F2AE102880BDE8B7
S315080021C0F08779480078012803D045F68960288089
S315080021D0F5E71EB945F6C3502880F0E71FB1B7F5F5
S315080021E0004F02D100E000BF03E045F625602880D5
S315080021F0E5E700BF6D493068884203D045F6C4500C
S315080022002880DCE700BF00BF4020FEF759F8824669
S3150800221000BF00BF96F82800B8B965480068706224
S31508002220012086F828000CB1F06A20603146604823
S31508002230006800F057FF00BF00BF5046FEF74EF893
S3150800224000BF00BF00202880B9E75949706A0968AD
S31508002250884221D196F82800FF280AD100BF00BF7E
S315080022605046FEF73BF800BF00BF45F28470288051
S31508002270A5E796F82800401C86F828000CB1F06AF5
S31508002280206000BF00BF5046FEF728F800BF00BF19
S3150800229045F28270288092E707F4004068B100BFD3
S315080022A000BF5046FEF71AF800BF00BF0CB1002069
S315080022B0206046F2B010288081E73E48007868B171
S315080022C000BF00BF5046FEF709F800BF00BF0CB1BB
S315080022D00020206046F66350288070E7D6F82480F0
S315080022E098F83B003249096891F83B10884206DDA8
S315080022F02F48006890F83B10404601F05DFB4B46BE
S3150800230004222B480168304600F042FF00BF00BF98
S315080023105046FDF7E3FF00BF00BF00F055F800BFC9
S3150800232000BF4020FDF7CCFF824600BF00BF204813
S31508002330006890F8390030B101280CD002281AD06C
S31508002340032821D110E01CB119480068C06C206030
S31508002350002028801CE01CB115480068C06C20606D
S3150800236046F2A910288013E00CB10020206047F23D
S31508002370D92028800CE01CB10D480068C06C20608C
S3150800238045F6C250288003E046F62E60288000BF36
S3150800239000BF00BF00BF5046FDF7A0FF00BF00BF4B
S315080023A000BF0CE794100020951000204D55545896
S315080023B030110020C210002010B5044600BFFEF7F9
S315080023C0A5F900BF10BD000010B50024224800780A
S315080023D0012800D010BD2148007800B1FAE720484E
S315080023E0007800B1F6E700BF4020FDF769FF044614
S315080023F000BF00F0F1FF1B4908700846007800EBA3
S315080024004000194951F82000184908600846006834
S3150800241017490968884205D100BF2046FDF75EFFC7
S3150800242000BFD7E711480068D0F89400401C0F4950
S315080024300968C1F894000F480068401C0D490860F7
S31508002440FEF713F900BF2046FDF748FF00BFBFF3AC
S315080024506F8F00BFBEE70000951000209410002083
S31508002460C2100020B71000203824002034110020A4
S3150800247030110020F010002070B504461C48007882
S31508002480012803D045F68B60208070BD00256D1CA1
S315080024906D1C6D1C17480088A84203DC45F68C6045
S315080024A02080F2E714480078E8B900F095FF134950
S315080024B0087008460078124908701048007800EB42
S315080024C04000104951F820000F4908600846006886
S315080024D00E490860012008490870FEF787F843F698
S315080024E09920208002E045F68A60208000BFCCE76C
S315080024F096100020F810002095100020B710002034
S31508002500B610002038240020341100203011002095
S315080025102DE9F04107464FF0000800BF00BF4020F4
S31508002520FDF7CEFE804600BF00BF00203B4908806D
S315080025303B4908603B4908603B4908603B490860DD
S315080025403B4908603B49088100BF00BF4046FDF78C
S31508002550C5FE00BF00BF00BF00BF4020FDF7B0FEAC
S31508002560804600BF00BF3448046800BF00BF40462D
S31508002570FDF7B4FE00BF00BF21E000BF00BF40204A
S31508002580FDF79EFE804600BF00BF002044F8800F7E
S31508002590E06260612082608220626062FEF7B8F8BD
S315080025A0E061803C04F16C060020B081D4F8BC40A0
S315080025B000BF00BF4046FDF791FE00BF00BF002CDC
S315080025C0DBD100BF00BF4020FDF77AFE804600BF82
S315080025D000BF1A48056800BF00BF4046FDF77EFEEB
S315080025E000BF00BF13E000BF00BF4020FDF768FE34
S315080025F0804600BF00BF05F120060020B081AD6906
S3150800260000BF00BF4046FDF769FE00BF00BF002DB2
S31508002610E9D100203880BDE8F0810000D6100020FE
S31508002620EC100020081100200C11002020110020B9
S31508002630241100202C240020F4100020BC100020B7
S31508002640704700002DE9FF4F85B004469346DDE943
S315080026501995DDE91286159F0020029062480078D8
S3150800266028B147F24A10288009B0BDE8F08F1CB996
S3150800267047F2AD102880F7E7BBF1000F03D147F208
S315080026804F102880F0E71EB946F62F602880EBE742
S3150800269056480068874203D246F630602880E3E74A
S315080026A01498B84203D346F631602880DCE7B8F1BF
S315080026B01E0F06D9B8F11F0F03D046F273202880E3
S315080026C0D2E7B8F11F0F06D14948844203D046F233
S315080026D073202880C8E7204601F02CFA00202880BD
S315080026E009F0010010B909F0020088B109F00200EA
S315080026F070B1B2460020049007E00020CAF8000036
S315080027000AF1040A0498401C04900498B842F4D3C9
S31508002710149806EB80000390CDE9007932465846B6
S31508002720039B089900F0B4F98246B24503D246F6EF
S315080027303260288098E73946304601F071FAC4F8C5
S3150800274024B00898A0620698E06084F83B8084F874
S315080027503C80C4F800A00398A0601798E065179815
S3150800276018B924480068206601E01798206618986A
S31508002770606026626764A4F8489004F16C001699B4
S3150800278000F090FC204600F03BF800BF00BF402058
S31508002790FDF796FD029000BF00BF94F83B0000F0DD
S315080027A031FE204600F08EFE204601F079F91248E7
S315080027B00088401C1049088010480078012807D076
S315080027C000BF00BF0298FDF789FD00BF00BF4BE7B9
S315080027D000BF00BF0298FDF781FD00BF00BFFFF7ED
S315080027E0F3FD00BF40E70000941000207454000871
S315080027F068230020C4100020F8100020951000203F
S31508002800704700002DE9F04104460E464FF00008D7
S315080028106148007820B147F24E103080BDE8F0815B
S315080028205E480078012803D045F689603080F5E7D0
S315080028305B48844203D147F24C103080EEE784B9F6
S3150800284000BF00BF4020FDF73BFD804600BF00BF2C
S315080028505448046800BF00BF4046FDF73FFD00BF6F
S3150800286000BF00BF00BF4020FDF72AFD804600BF1D
S3150800287000BF94F83A0008285ED2DFE800F00409A1
S315080028800E10080A0F11204600F03AFE5FE05EE0DF
S3150800289000BF204601F07AFA59E000BF00BF00BF2A
S315080028A094F83800082839D2DFE800F0040705381C
S315080028B00D08090600BF00BF31E000BF00BF204673
S315080028C000F00DFD2BE0606B456A15F83B7F20464E
S315080028D000F005FD287869783B3D884212D095F8C6
S315080028E03B0094F83B1088420CD1284600F02DFC9A
S315080028F0074695F83C00B84202DA95F83C0000E035
S3150800290038460746002084F8380095F83B00B84258
S3150800291003D03946284601F04FF800E000BF00BF53
S3150800292094F83A00032803D094F83A00072802D10D
S31508002930204601F02BFA0AE000BF00BF4046FDF72B
S31508002940CDFC00BF00BF46F62D60308066E700BFAD
S31508002950206C10B1204600F0C9FB04F16C0000F0B1
S3150800296081FB204600F022F8204601F0B1F80E4817
S315080029700088401E0C490880FF2084F83A00002091
S31508002980308000BF00BF4046FDF7A8FC00BF00BF6F
S31508002990FFF71AFD00BF41E79410002095100020AC
S315080029A06823002030110020F81000207047704777
S315080029B02DE9F05F05460E4617461C464FF0000BFC
S315080029C03148007820B147F259102080BDE8F09FC1
S315080029D01EB946F2D5202080F8E71FB946F2D52061
S315080029E02080F3E700BF00BF4020FDF769FC83465F
S315080029F000BF00BF0DB925480568286868B900BF3B
S31508002A0000BF5846FDF76AFC00BF00BF00203060D3
S31508002A10386047F252102080D8E795F8480000F051
S31508002A20010068B900BF00BF5846FDF757FC00BF54
S31508002A3000BF00203060386047F254102080C5E798
S31508002A40D5F820A00AF1200AD5F8449000BF00BFA7
S31508002A505846FDF743FC00BF00BF4FF0000803E0EF
S31508002A600AF1040A08F10108C84503D2DAF8000099
S31508002A700028F5D0C6F80080A9EB080038600020C9
S31508002A80208000BFA2E7000094100020301100202B
S31508002A90F0B50446DDE9055602EB850020F007008F
S31508002AA04FF0807C071F3846C7F800C0071F384616
S31508002AB03C60DFF8A8C0071F3846C7F800C04FF0CB
S31508002AC0123C071F3846C7F800C04FF0033C071FE3
S31508002AD03846C7F800C04FF0023C071F3846C7F80B
S31508002AE000C0071F38463B60071F384639606FF03D
S31508002AF0020C071F3846C7F800C04FF0113C071FE5
S31508002B003846C7F800C04FF0103C071F3846C7F8CC
S31508002B1000C04FF0093C071F3846C7F800C04FF001
S31508002B20083C071F3846C7F800C04FF0073C071F88
S31508002B303846C7F800C04FF0063C071F3846C7F8A6
S31508002B4000C04FF0053C071F3846C7F800C04FF0D5
S31508002B50043C071F3846C7F800C0F0BDE13B000833
S31508002B6030B504460CB90B480468216A20688842C7
S31508002B7006D3616C206A00EB81002168884201D87F
S31508002B80002030BD616C206A01F036F805462846FB
S31508002B90F7E700003011002070B5FDF7B9FD0546CE
S31508002BA01548006815490968884215D01248006812
S31508002BB0D0F89C00281A10490968C1F898000E48F0
S31508002BC00068D0F8A0000C490968D1F898100844A4
S31508002BD009490968C1F8A00008480068C0F89C506F
S31508002BE00020FFF7BDFF0446012C03D00248006809
S31508002BF0FFF7E2FB70BD0000301100203411002001
S31508002C002DE9F04106460D46144600272748007868
S31508002C1020B147F275202080BDE8F081244800786D
S31508002C20012803D045F689602080F5E72148007819
S31508002C3018B146F663502080EEE735B1022D05D06F
S31508002C40042D05D0082D04D101E000BF00BF00BF48
S31508002C5003E045F625602080DEE700BF00BF00BF21
S31508002C604020FDF72DFB074600BF00BF23462A4636
S31508002C7031461148006801F043F8208838B100BF92
S31508002C8000BF3846FDF72AFB00BF00BFC4E70A4865
S31508002C90006800F035FC00BF00BF3846FDF71EFB94
S31508002CA000BF00BFFFF790FB00BFB5E794100020F8
S31508002CB095100020C21000203011002070B504467F
S31508002CC0002600BF00BF4020FDF7FAFA064600BFFF
S31508002CD000BF0648056800BF00BF3046FDF7FEFA8C
S31508002CE000BF00BF00202080284670BDFC100020D1
S31508002CF00EB5474802904748009047480290474813
S31508002D000290474800904748029047480190474834
S31508002D100290474802904748029047480290474821
S31508002D200190474801904748019047480290474814
S31508002D300190474802904748019047480190474804
S31508002D4001904748019047480290474802904748F3
S31508002D5002904748019047480290474802904748E2
S31508002D6001904748019047480190474801904748D5
S31508002D7001904748019047480290474802904748C3
S31508002D8002904748029047480190474801904748B3
S31508002D9001904748029047480290474802904748A2
S31508002DA00190474801904748019047480090474896
S31508002DB00190474802904748029047480290474882
S31508002DC00290474802904748029047480290474871
S31508002DD00190474802904748029047480190474863
S31508002DE00190474802904748029047480190474853
S31508002DF00190474802904748029047480190474843
S31508002E0001900298029001980190009800900EBDDA
S31508002E1098540008FC550008995400089A5400086C
S31508002E209C540008A0540008A4540008A1540008A3
S31508002E30CC540008CD540008CE540008D0540008DD
S31508002E40D2540008D4540008F4540008F654000874
S31508002E50F8540008FA540008FC540008FE54000808
S31508002E60005500083055000831550008325500084D
S31508002E7034550008365500083755000838550008F7
S31508002E803A5500083C5500083E55000840550008CC
S31508002E90445500087455000875550008765500080D
S31508002EA077550008785500087A5500087C550008BB
S31508002EB0A4550008A5550008A6550008A7550008FA
S31508002EC0A8550008AA550008AC550008B0550008D2
S31508002ED0B1550008B2550008B3550008B4550008A6
S31508002EE0B5550008B6550008B7550008B855000886
S31508002EF0BA550008BB550008BC550008BE55000861
S31508002F00C0550008C1550008C2550008C455000838
S31508002F10F4550008F5550008F6550008F855000858
S31508002F20002400BF00BF00BF4020FDF7C9F90446D2
S31508002F3000BF00BF08480068401C074908600748EA
S31508002F400068401C0549086000BF00BF2046FDF721
S31508002F50C5F900BFE6E7000090100020D810002051
S31508002F6010B58AB0044600200E4908600B200021DF
S31508002F700591CDE90704069108460B4909680B4AED
S31508002F8012680B4B1B68CDE90132CDE903101F20EF
S31508002F900023084A08A100900C48FFF753FB0AB023
S31508002FA010BD0000901000203C540008385400085A
S31508002FB034540008212F000875432F4F532D4949D3
S31508002FC0492049646C65205461736B0068230020AE
S31508002FD00021034A1160034A1180018070470000EE
S31508002FE0A8100020AC10002070B501461A4D2D68B7
S31508002FF01DB945F21E750D8070BD184D2D881DB979
S3150800300045F21D750D80F7E7134D28682A681032BA
S31508003010124D2D886D1EACB2002308E00260002513
S3150800302045600581C560103010325D1CABB2A34205
S31508003030F4DB0025056045600581C560064D2D68F1
S31508003040074E3560054D2D88B5800025F5803581FC
S315080030500D8000BFD0E700005854000850540008FF
S315080030602C24002010B5014648894B89BBB10A6853
S315080030700B4B1B6813600A4C4B6823602346DB889E
S315080030804C891B1B064CE38023469B884C892344AA
S31508003090034CA38000234B818B810B604B6010BDD2
S315080030A02C24002001810022428182810260426034
S315080030B07047000009A1C1610021416108490968FA
S315080030C011B90021816105E0054909688161044952
S315080030D0096848610249086070470000200000003E
S315080030E0B0100020026C0A62016470472DE9F843AB
S315080030F005462C6C25E0D4F82090FDF709FB8046A0
S31508003100C4F82C802146284600F034F804F1080655
S31508003110306820B9002084F82800606210E037681B
S315080031206562012084F8280021463846FFF7DAFF51
S3150800313000231A4639462046CDF8008000F0F6F8F6
S315080031404C46002CD7D1BDE8F88330B504461F207D
S3150800315004F140010AE00D68AB6823B193F83B20FF
S31508003160824200DA10460D6805F120010D68002D2F
S31508003170F1D130BD024602F1400002E0036803F1D6
S31508003180200003688B42F9D103681B6A0360704705
S315080031902DE9F04105460C4616461F4684F8386068
S315080031A0002084F839003946204600F0EDFB3DB191
S315080031B005F1080865632146404600F05DF801E020
S315080031C0002060632146284600F002F8BDE8F08139
S315080031D010B540B14468C1F8C04000F108031A6848
S315080031E0D468C46113E091F83840022C02D0072C49
S315080031F008D103E006A4C1F8C04007E006A4C1F858
S31508003200C04003E007A4C1F8C04000BF00BF10BD1E
S315080032105461736B205100005461736B2053656DC4
S31508003220000000002000000010B50A4606A4C2F8F7
S31508003230C04040B100F10803196811B1CC68C461F7
S3150800324001E001A4C46110BD2000000070B5044669
S31508003250666B06F108052868C06A38B1204600F092
S315080032603EF866632146284600F006F870BD002140
S31508003270016041600181704710B591F83B300468E0
S315080032803CB9012404810024CC620C6301604160CE
S3150800329024E00489641C0481026805E092F83B4036
S315080032A09C4200DD02E0D26A002AF7D100BF3AB993
S315080032B00024CC6244680C630C6BE16241600DE04B
S315080032C0146B2CB9CA6200240C631163016005E013
S315080032D0CA62146B0C630C6BE162116310BD10B506
S315080032E0446B14B3446B04F108010C68E46A1CB916
S315080032F000240C604C6011E0046B24B9C26A0024F7
S3150800330014630A600AE0C46A24B9036B0024DC6209
S315080033104B6003E0036BC26ADA6213630C89641EAE
S315080033200C810024C4620463446310BD2DE9F04196
S3150800333005460C4616461F46DDF8188094F83A00EE
S31508003340082845D2DFE800F00405080906072728FB
S3150800335000BF00BF00BF3CE000BF6666A4F8687007
S31508003360C4F84C8015B12046FFF7B9FF2146284618
S31508003370FFF75AFF94F83A00032802D1204600F0D6
S3150800338005FD204600F068F800203834A07060700B
S3150800339004F838091DE000BF6666A4F86870C4F82A
S315080033A04C8015B12046FFF79AFF21462846FFF7BD
S315080033B03BFF94F83A00072802D1204600F0E6FCC5
S315080033C004203834A0700020607004F8380900E042
S315080033D000BF00BFBDE8F08110B503490868FCF7D7
S315080033E08AFFC0B210BD0000B8100020002004E01B
S315080033F00021034A42F82010401C0028F8D07047E4
S31508003400B810002004490968C0F11F0301229A4038
S315080034101143014A11607047B81000200449096831
S31508003420C0F11F0301229A409143014A1160704777
S31508003430B8100020002109E001EB4102054B03EB1F
S3150800344082000022028102604260491C2029F3D3CF
S31508003450704700003824002010B5044694F83B0055
S31508003460FFF7D0FF94F83B0005490978884203D155
S31508003470204600F027F802E0204600F003F810BDC9
S31508003480B610002010B590F83B3003EB43030C4C04
S3150800349004EB83010B683BB901230B81002303610D
S315080034A043610860486009E00B895B1C0B810B6867
S315080034B00361002343610A685061086010BD00007B
S315080034C03824002010B590F83B3003EB43030B4C2F
S315080034D004EB83010B683BB901230B8100230361CD
S315080034E043610860486008E00B895B1C0B81002378
S315080034F003614A6842611061486010BD38240020A3
S315080035002DE9F041054695F83B0000EB40001249CD
S3150800351001EB80046F692E6987B946B900202081BE
S315080035202060606095F83B00FFF778FF0EE0208981
S31508003530401E208100207061266007E02089401E19
S3150800354020813E610EB9676000E0776100206861FE
S315080035502861BDE8F08100003824002088B00020EA
S31508003560009006E0BD490968480002AA0021FFF755
S3150800357047FBBB4800780128F4D102A8FEF7C8FF2C
S315080035804FF00008B7480068B4490968884205D969
S31508003590B4480068B1490968B0FBF1F8B8F1000F02
S315080035A004D1B04800680A21B0FBF1F800BFFDF766
S315080035B0AFF8814600BF00BF4020FCF781FE0090AF
S315080035C000BF00BFA8480068A84908600020A649AF
S315080035D0086000BF00BF0098FCF780FE00BF00BF70
S315080035E0A3480068A1490968884248D9A0480068E4
S315080035F0A049884205D242F2107004900120039037
S3150800360023E09B4800689C49884205D24FF47A70AB
S3150800361004900A20039018E0954800689749884264
S3150800362003D26420049003900FE0914800689449FF
S31508003630884205D20A2004904FF47A70039004E079
S315080036400120049042F2107003908948016803989B
S31508003650B1FBF0FB8549049809684843B0FBFBF0C9
S3150800366042F21071081A8749088087480088098835
S31508003670884207DA834800888349088002E00020E8
S3150800368080490880FEF7DCFF002500BF00BF402008
S31508003690FCF716FE009000BF00BF7C48046800BF18
S315080036A000BF0098FCF71AFE00BF00BF28E000BF65
S315080036B000BF4020FCF704FE009000BF00BF54F88E
S315080036C0A00F6060002044F8A00900BF00BF009862
S315080036D0FCF704FE00BF00BFD4F8A400054400BFF1
S315080036E000BF4020FCF7ECFD009000BF00BFD4F8F7
S315080036F0BC4000BF00BF0098FCF7F0FD00BF00BF4C
S31508003700002CD4D15DB35B48854205D242F21070D5
S315080037100690012007901DE05748854205D24FF4D0
S315080037207A7006900A20079014E05448854203D21E
S315080037306420069007900DE05148854205D20A207C
S3150800374006904FF47A70079004E00120069042F242
S31508003750107007900798B5FBF0F0059003E000207D
S3150800376006900120059000BF00BF4020FCF7A8FD89
S31508003770009000BF00BF4548046800BF00BF00981E
S31508003780FCF7ACFD00BF00BF2CE0D4F8A4000699F6
S3150800379048430599B0FBF1F086B242F210708642B2
S315080037A000D90646A4F89060B4F89200B04201DA4F
S315080037B0A4F8926002AB04F1B002111D2046FFF78F
S315080037C0F7F800BF00BF4020FCF77AFD009000BF65
S315080037D000BFD4F8BC4000BF00BF0098FCF77EFDD0
S315080037E000BF00BF002CD0D100272948D0F800A080
S315080037F00AF1200A274800680838019002E00AF111
S31508003800040A7F1CDAF8000010B901988742F6D33B
S31508003810214807601F480068C01B204908602048E7
S315080038200078012805D100201D49087002A8FEF776
S315080038306FFEFCF76DFFA0EB09001A4908601A48ED
S3150800384000680968884203D2164800681649086065
S3150800385002AA00214046FFF7D3F9A8E660540008FB
S31508003860E410002078540008D8100020E01000204A
S31508003870DC100020801A060000093D00005A62028A
S315080038800084D717D4100020D6100020F41000208A
S315080038904454000848540008981000209C10002042
S315080038A0D2100020E8100020EC10002010B58AB0D5
S315080038B0044600202149086021490860214908601A
S315080038C02149087021490870214908602149086082
S315080038D02148006820B946F62B6020800AB010BD42
S315080038E01E4800681E490968884203D246F62C60BD
S315080038F02080F3E71B4800781F2803D346F62A6082
S315080039002080EBE7032000210591CDE90704069105
S31508003910084612490A68144909680F4B1B68CDE91D
S315080039200131CDE903200F48007800230F4A10A182
S3150800393000901448FEF786FE00BFCFE7D810002097
S31508003940E0100020DC100020E4100020D210002037
S31508003950981000209C100020645400086C5400083D
S31508003960745400085C540008685400085D35000863
S3150800397075432F4F532D4949492053746174205478
S3150800398061736B00B825002070B504460D4655B125
S315080039902B46084800210268204600F05BF9032000
S315080039A084F83A0002E0022084F83A002046FFF73D
S315080039B0A7FD70BDFC1000202DE9F04104460D4618
S315080039C000BF002694F83B7094F83A0008285DD2A8
S315080039D0DFE800F004191E1F1A1B20212046FFF7F6
S315080039E08FFD84F83B5094F83B00FFF70BFD2B48FE
S315080039F00068844203D12046FFF744FD02E02046D2
S31508003A00FFF760FD44E000BF00BF84F83B503FE08D
S31508003A1000BF00BF00BF84F83B5094F83800082860
S31508003A202FD2DFE800F02E042F2E0A05063000BF3D
S31508003A3000BF2046FFF70AFC26E02046FFF706FCF3
S31508003A40606B466AAF4205DD96F83B00A84217DC74
S31508003A50002615E096F83B00B84211D13046FFF72C
S31508003A6074FB054696F83C00A84202DA96F83C0034
S31508003A7000E02846054696F83B00A84200D10026F5
S31508003A8002E000BF00BF00BF00BF01E0BDE8F08153
S31508003A9000BF3446002C94D100BFF7E73011002050
S31508003AA00021C0F8B8100949096819B90021C0F8F9
S31508003AB0BC1007E005490968C0F8BC100349096845
S31508003AC0C1F8B8000149086070470000F4100020EA
S31508003AD0D0F8B820D0F8BC104AB90D4B196011B10E
S31508003AE00023C1F8B8300023C0F8BC300FE029B96C
S31508003AF00023C2F8BC30C0F8B83008E0C2F8BC10E1
S31508003B00C1F8B8200023C0F8BC30C0F8B8307047F8
S31508003B10F41000200021044A1160044A1180044A66
S31508003B201160018070470000F4100020F810002092
S31508003B30F010002010B5044600202060A0606060E8
S31508003B4020616061A061E06122A0E060002020623F
S31508003B506062A062E0646066A4F86800002104F16F
S31508003B606C00FFF79FFA00202C3420656065A0657D
S31508003B70A4F86000E0656062E067C4F88000A061B0
S31508003B8084F86200C4F88800C4F88400A083A062A0
S31508003B90E06220636063A4F86400A4F86600A06687
S31508003BA0E066FCF7B5FD206700206067206060606E
S31508003BB0A06020736073A0732020E0732074002037
S31508003BC06061C4F88C00C4F8900004A0C4F894009E
S31508003BD02C3C10BD3F5461736B00000020000000B0
S31508003BE008B504480068FEF7E2FE69460020FEF7BD
S31508003BF009FE08BD3011002010B502460B4600210B
S31508003C0007E0064C1068A04201D0002010BD121D26
S31508003C10491C0829F5D30120F8E700004523CDAB58
S31508003C200246002003E0034B42F82030401C0828D7
S31508003C30F9D370474523CDAB00210180034A1160B3
S31508003C40034A11609180D18070470000FC10002063
S31508003C50001100202DE9F04304460F469446984685
S31508003C6008EB0C00DFF89090D9F80090B944A0EB67
S31508003C7009021AB900206065BDE8F0831F4B186871
S31508003C8038B962650020A061E0611C600120988057
S31508003C90F2E79888401C98801968486DC61BB2429E
S31508003CA00BD2C86948B96265B01A48650020E06158
S31508003CB0A161CC611C600120DEE7921B0D46A96953
S31508003CC003E0486D121A0D46896911B1486D904294
S31508003CD0F7D949B1CD696265E561A161486D801A78
S31508003CE04865CC61AC6104E06265E5610020A061CD
S31508003CF0AC610120C0E70000FC1000200011002084
S31508003D002DE9F04F06460C4691461F464FF0000B2C
S31508003D10B9F1040F01D1002520E0B9F1080F1BD134
S31508003D2024B947F27E203880BDE8F08FB56D164875
S31508003D300068A0EB0508A0450AD3B8FBF4F004FB1D
S31508003D400055B8FBF4F004FB108000B12544B565B6
S31508003D50B06D2044B06501E00B48056823462A4645
S31508003D6059463046FFF776FF8246BAF1010F05D16C
S31508003D70012086F83A000020388002E047F27E20CB
S31508003D80388000BFD0E70000FC10002030B5C369BA
S31508003D908169134A9BB921B900241460948044654B
S31508003DA01CE00024CC614C6D456D2C444C651160BB
S31508003DB09488641E94800024846144650EE09961A9
S31508003DC021B1CB614C6D456D2C444C650024C46112
S31508003DD09488641E948000248461446530BD000084
S31508003DE00011002010B5002400BF00BF4020FCF7DA
S31508003DF067FA044600BF00BF084809490860094831
S31508003E00086201F10800FFF732FA00BF00BF20463A
S31508003E10FCF764FA00BF00BF10BD0000434F4E44D4
S31508003E207C260020A0260020F8B5002600BF00BF8B
S31508003E304020FCF745FA064600BF00BFFCF768FCC1
S31508003E4004460F48C4620F4D286838B900BF00BF42
S31508003E503046FCF743FA00BF00BFF8BD00231A46F8
S31508003E600949084808380094FFF760FA00BF00BF00
S31508003E703046FCF733FA00BF00BF00BFEDE700008D
S31508003E80A026002084260020D02600202DE9F8430D
S31508003E9007464FF0000800BF00BF4020FCF710FAA5
S31508003EA0804600BF00BFFCF733FC06463F48C662A3
S31508003EB001463F48FFF75EF93C4D08353C4890F807
S31508003EC03B003B4991F83C1088420AD0384890F8A4
S31508003ED03C00374981F83B00084690F83C003549D4
S31508003EE00870286828B900203049486281F82800F7
S31508003EF010E02C682D48446201202C4981F82800DE
S31508003F002046FFF7EFF800231A4621462748009671
S31508003F10FFF70CFA3B46032225492748FFF738F9ED
S31508003F2000BF00BF4046FCF7D9F900BF00BFFEF747
S31508003F304BFA00BF00BF4020FCF7C2F9804600BF1D
S31508003F4000BF1A48406A80B918491948FFF7CAF8E5
S31508003F50174816494862012081F8280000BF00BFAB
S31508003F604046FCF7BBF900BF1DE01048446A94F8C8
S31508003F703B000F4991F83B10884205DD0C4890F844
S31508003F803B102046FFF718FD00230422084907487E
S31508003F90FFF7FEF800BF00BF4046FCF79FF900BFD9
S31508003FA000BFFEF711FABDE8F8830000A02600203E
S31508003FB0D0260020B61000207C26002010B58AB036
S31508003FC0044600202A4908802A4908602A490860C8
S31508003FD02A4908802A4800682A490968B0FBF1F08E
S31508003FE029490860002029490860294908602246AD
S31508003FF028A12C48FEF784F8208808B10AB010BD1D
S31508004000FFF7F0FE2848006818B947F247302080C5
S31508004010F4E72648006826490968884203D247F229
S3150800402048302080EAE7234800781F2803D347F260
S3150800403046302080E2E70B20002105910A46CDE9AB
S3150800404007040691194800681B490968164B1B683E
S31508004050CDE90131CDE90302164800780023174A55
S3150800406017A100901C48FEF7EDFA00BFC6E700004E
S315080040701C11002010110020181100201411002016
S3150800408078540008805400082C11002020110020C4
S31508004090241100204F5320546D72204D7574657895
S315080040A000000000A0260020845400088C54000854
S315080040B0745400087C54000888540008AD41000870
S315080040C075432F4F532D4949492054696D65722010
S315080040D05461736B00000000D02600202DE9F047DC
S315080040E0054688462848006870B900202861686136
S315080040F0254805600120254908802548C0F8008024
S31508004100FFF792FEBDE8F08720480088401C1F494B
S315080041100880A86940441E490968461A1A4804686E
S31508004120D4F818904E4510D2606970B9A9EB06000C
S31508004130A061002068612C61656113480560144818
S31508004140C0F80080FFF770FEDCE7A6EB09062746F5
S315080041503C6903E0A069361A2746246914B1A069A8
S31508004160B042F7D94CB16769AE616F612C61A0693D
S31508004170801BA06165613D6104E0AE616F6100204E
S3150800418028613D6100BFBDE7181100201411002009
S31508004190281100201CB501A800231A4619460090CC
S315080041A00148FDF7FDFF1CBDA02600204FF0000AC0
S315080041B0FFF7F0FF00BF3D48006810B94FF000094F
S315080041C003E03A480068D0F818904846FFF75EFEC4
S315080041D03648006800B9EEE7FCF79AFA804600BF51
S315080041E000BF4020FCF76CF8824600BF00BF30488D
S315080041F0076800BF00BF5046FCF770F800BF00BF55
S315080042002C4800683D1A2B480760284804680CE0CB
S31508004210A069A84204D2A0692D1A0020A06103E073
S31508004220A069401BA061002524690DB1002CEFD1BF
S315080042301E48046826E0042084F82600A66816B1FD
S315080042402046E168B04794F82600042818D1194892
S315080042500168204600F034F8A08C022809D184F8B9
S315080042602600206AA061134801682046FFF736FF3A
S3150800427006E0002060612061A061032084F8260022
S315080042800A48046814B1A0690028D4D0FCF740FA9B
S31508004290A0EB0800084908600848006809688842D1
S315080042A003D2054800680549086084E7181100200C
S315080042B0FC100020281100202011002024110020C5
S315080042C02DE9F04105460F46D5F814802C69B8F15A
S315080042D0000F40D154B900202949086029490880AF
S315080042E0A86129480760FFF79FFD46E02548008832
S315080042F0401E24490880244800683E1A0020606150
S31508004300A069A9690844A0611D4804600EE0A06977
S31508004310B04204D2A069361A0020A06103E0A06961
S31508004320801BA0610026A046D8F810400EB1002CCC
S31508004330EDD1134800688069A969884203D11048FD
S315080043400068806918B910480760FFF76DFD0020FE
S315080043502861A86111E00B480088401E09490880B9
S31508004360C8F810402CB1C4F81480A069A96908449B
S31508004370A061002068612861A861BDE8F08100009D
S315080043801811002014110020281100202DE9F041F1
S3150800439004460D4616460E4F00BF387808B900F099
S315080043A0E3FB00BFEFF311800746202080F3118856
S315080043B000BF00BF32462946204600F00BF880466B
S315080043C0F8B280F3118800BF00BF4046BDE8F0810F
S315080043D0501600202DE9F047074688461646C2467D
S315080043E007EB47011B4800EBC109D9F8140020B1B7
S315080043F0012811D0022826D11EE0484600F0ECFB21
S315080044000546B54201D2002405E0344632465146F7
S31508004410484600F038FD18E0484600F0DDFB054642
S31508004420B54201D2284600E03046044622465146A7
S31508004430484600F028FD08E032465146484600F056
S31508004440E7FC044601E0002400BF00BF2046BDE8A3
S31508004450F0870000681600200FB438B5044606A891
S3150800446000906A462046059900F007F805460020A0
S315080044700090284638BC5DF814FB2DE9F04F99B03A
S3150800448082460D46144603A8149040201590002035
S315080044901690CDF860A0179000BF2E786D1C06B94F
S315080044A0DDE0252E79D100274FF0010900BF2E78CF
S315080044B0232E12D02B2E0CD02D2E02D0302E10D11A
S315080044C003E047F001076D1C0EE047F002076D1C7C
S315080044D00AE047F004076D1C06E047F008076D1C64
S315080044E002E04FF0000900BF00BFB9F1000FDED1AE
S315080044F04FF0000800BF2E78302E01DB392E00DD84
S3150800450007E06D1CA6F1300008EB880100EB4108B6
S31508004510F1E700BF002013902E782E2E12D16D1CC5
S3150800452000BF2E78302E01DB392E00DD09E06D1C28
S31508004530A6F13000139901EB810100EB41001390BD
S31508004540EFE700BF2E7800BF6C2E01D0682E02D18F
S315080045506D1C2E7800E000E0F6E700BF702E5DD0F7
S3150800456008DC252E6AD0582E35D0632E09D0642E45
S3150800457069D113E0732E3CD0752E1DD0782E62D1EA
S3150800458028E02168081D2060D1F8009009F0FF0B8B
S31508004590594614A800F01AFC56E058E02168081D90
S315080045A02060D1F80090CDE900870A22494614A870
S315080045B0139B00F01FFB47E02168081D2060D1F817
S315080045C00090CDE900870A22494614A8139B00F0FB
S315080045D087FB39E000BF2168081D2060D1F80090EC
S315080045E0CDE900871022494614A8139B00F078FBF2
S315080045F02AE02168081D2060D1F800B000BF9BF8AA
S3150800460000600BF1010B06B906E0314614A800F06C
S31508004610DDFB17980028F2DA00BF15E02168081DAF
S315080046202060D1F80090002008210B461022CDE921
S315080046300010494614A800F053FB05E0252114A8EC
S3150800464000F0C4FB00E000BF00BF6D1C03E031466C
S3150800465014A800F0BBFB17980028BFF61EAF00BFD2
S31508004660179800280ADD169820B103A95046169A0D
S31508004670FFF78CFEDDE9161008441790179819B055
S31508004680BDE8F08F704700000348006840F47000EA
S31508004690014908607047000088ED00E070B50546DE
S315080046A0AC6B0020E085E0842046FCF7E6FF70BD91
S315080046B00168C96821F490710268D1600168496986
S315080046C021F0010102685161016B012905D10168D8
S315080046D0C96821F010010268D160202180F83E10D7
S315080046E000210163704710B504462068C06820F0B1
S315080046F040002168C860202084F83D002046FDF768
S3150800470089F9002010BD70B5044694F83E002228A9
S3150800471056D1A068B0F5805F0CD1206950B9002544
S31508004720A66A20684068C0F308003080A06A801C2A
S31508004730A06215E0A56A0026A068B0F5805F03D0E0
S31508004740A06828B9206918B920684068287004E06C
S315080047502068406800F07F002870A06A401CA062AC
S31508004760E08D401E80B2E08540BB2068C06820F01E
S3150800477020002168C8602068C06820F4807021681D
S31508004780C8602068406920F001002168486120203F
S3150800479084F83E00206B01280AD12068C06820F002
S315080047A010002168C860A18D2046FCF765FF02E06D
S315080047B02046FDF7F1F80020206370BD0020FCE7D5
S315080047C00220FAE72DE9F84F04462068006920F42C
S315080047D04050E1680843216808612169A0680843D8
S315080047E061690843E169084300902068C06849F296
S315080047F00C618843009908432168C86020684069AD
S3150800480020F44070A1690843216848617649206808
S31508004810884203D075492068884203D1FCF748FCD2
S31508004820814602E0FCF734FC8146E069B0F5004FAA
S315080048306CD102206168A0FB015003461920A9FB30
S31508004840007001462A463846FBF761FD6421B0FB35
S31508004850F1F04FEA001A02206168A0FB01510B46ED
S315080048601920A9FB00712A463846FBF750FD8346F6
S3150800487002206168A0FB015003461920A9FB0071BC
S315080048802A463846FBF743FD6421B0FBF1F000EBFE
S31508004890C00101EB0010ABEB8000322101EBC00038
S315080048A06421B0FBF1F000F0F8000AEB400A0220A0
S315080048B06168A0FB015003461920A9FB0070014658
S315080048C02A463846FBF723FD834602206168A0FB8B
S315080048D0015003461920A9FB00712A463846FBF702
S315080048E016FD6421B0FBF1F000EBC00101EB0010EE
S315080048F0ABEB8000322101EBC0006421B0FBF1F084
S3150800490000F007005044216888606AE00420616866
S31508004910A0FB015003461920A9FB007001462A4650
S315080049203846FBF7F4FC824604206168A0FB015078
S3150800493003461920A9FB007001462A463846FBF7AC
S31508004940E6FC6421B0FBF1F000EBC00101EB0010BE
S31508004950AAEB8000322101EB00106421B0FBF1F0D4
S3150800496000F0F00A04206168A0FB017003461920D4
S31508004970A9FB00513A462846FBF7C9FC6421B0FB5F
S31508004980F1F00AEB001A04206168A0FB01510B46FE
S315080049901920A9FB00712A463846FBF7B8FC83465E
S315080049A004206168A0FB015003461920A9FB00708A
S315080049B001462A463846FBF7AAFC6421B0FBF1F00B
S315080049C000EBC00101EB0010ABEB8000322101EBDC
S315080049D000106421B0FBF1F000F00F00504421688C
S315080049E08860BDE8F88F00000010014000140140FF
S315080049F010B5034699629A85DA8500201864222044
S31508004A0083F83E0000BF002083F83C0000BF18680A
S31508004A10C06840F480701C68E0601868406940F01F
S31508004A2001001C6860611868C06840F020001C68B6
S31508004A30E060002010BD014691F83D00212828D1EC
S31508004A408868B0F5805F0BD1086948B90A6A10888A
S31508004A50C0F308000B685860086A801C086205E005
S31508004A600B6A581C086218780B685860C88C401E78
S31508004A7080B2C88458B90868C06820F080000B68FE
S31508004A80D8600868C06840F040000B68D86000200D
S31508004A9070470220FCE7000070B500242C4D2D4815
S31508004AA0FCF7F6FD00BF03E0641CAC4200D904E045
S31508004AB02848FCF7E3FD2028F6D100BF002403E0D0
S31508004AC0641CAC4200D906E0012223492148FCF7C0
S31508004AD041FF0028F4D100BF2048FCF7D9FD002487
S31508004AE003E0641CAC4200D904E01C48FCF7C6FD90
S31508004AF02028F6D100BF002403E0641CAC4200D98C
S31508004B0006E0012214491548FCF724FF0028F4D1D1
S31508004B1000BF1348FCF7BCFD002403E0641CAC424C
S31508004B2000D904E00E48FCF7A9FD2028F6D100BFFD
S31508004B30002403E0641CAC4200D906E001220649C1
S31508004B400748FCF707FF0028F4D100BF70BD000036
S31508004B50FFFF0100001200206A0E00204412002008
S31508004B608812002000BFFEE710B5124C0220206113
S31508004B70606111A0A0611349E1614FF4806121626F
S31508004B800021A1626162E1620BA0A0640E49E164A2
S31508004B90102121650021A1656165E1650BA1E01D74
S31508004BA0FBF72CFC0AA12046FBF728FC2020A07165
S31508004BB010BD0000501600205465726D696E616C58
S31508004BC000000000C8160020C81A002052545400DD
S31508004BD0534547474552000010B501460A69CB6858
S31508004BE09A4204D88C68641EE41AA01801E0D41A04
S31508004BF0601E10BD2DE9FC5F06460F469246984694
S31508004C00DDE90C45002F01DA784200E03846834694
S31508004C104FF0010903E09BFBFAFB09F10109D345B3
S31508004C20F9DAC84500D9C14634B1002F03DB05F0CF
S31508004C300400042800D1641E05F0020010B1B8F182
S31508004C40000F11D005F0010070B96CB108E0641EC0
S31508004C502021304600F0BAF8F068002800DA02E0B1
S31508004C600CB1A145F3D300BFF068002836DB002F4E
S31508004C7005DA7F422D21304600F0A8F807E005F056
S31508004C800400042803D12B21304600F09FF8F06871
S31508004C90002823DB05F00200022814D105F00100E4
S31508004CA088B9B8F1000F0ED16CB108E0641E302146
S31508004CB0304600F08BF8F068002800DA02E00CB104
S31508004CC0A145F3D300BFF068002807DB43465246E8
S31508004CD039463046CDE9004500F002F8BDE8FC9FAC
S31508004CE02DE9FC5F8046894615461E460C9CCDF884
S31508004CF004900127BB4605E00198B0FBF5F001904A
S31508004D000BF1010B0198A842F6D25E4500D9B346CD
S31508004D100D9800F00100D0B9CCB10D9800F0020052
S31508004D20022803D116B93020009001E02020009017
S31508004D3009E0641E4046009900F048F8D8F80C00CF
S31508004D40002800DA02E00CB1A345F2D300BFD8F878
S31508004D500C00002835DB09E0012E01D9761E04E097
S31508004D60B9FBF7FAAA4500D201E06F43F4E700BFA2
S31508004D7000BFB9FBF7FA0AFB1799134810F80A108F
S31508004D80404600F023F8D8F80C00002800DA03E0C3
S31508004D90B7FBF5F7002FECD100BF0D9800F0010026
S31508004DA078B174B109E0641E2021404600F00EF87F
S31508004DB0D8F80C00002800DA02E00CB1A345F2D3BB
S31508004DC000BFBDE8FC9F00002454000870B50446E7
S31508004DD00E46A568681C6168814206D32068465558
S31508004DE0681CA060E068401CE060D4E901108842B5
S31508004DF00DD1A26821682069FFF7C8FAA168884220
S31508004E0003D04FF0FF30E06001E00020A06070BDE5
S31508004E102DE9F05F0446894617464FF0000AE56813
S31508004E2000BFD4F81080A84503D9A8EB0500461E94
S31508004E3004E0A5EB0800401CA1680E1AA068401BF8
S31508004E40B04201D9304601E0A068401B0646BE4282
S31508004E5001D2304600E038460646606800EB050B8E
S31508004E60324649465846FBF7EDFAB244B144BF1BF1
S31508004E703544A068A84200D10025E560002FD0D1AE
S31508004E805046BDE8F09F2DE9F04704468946154689
S31508004E90E668A068871BAF420AD9606800EB060A75
S31508004EA02A4649465046FBF7CDFA7019E06014E0E9
S31508004EB0B846606800EB060A424649465046FBF784
S31508004EC0C1FAA5EB0708D4F804A009EB0701424686
S31508004ED05046FBF7B7FAC4F80C80BDE8F087000027
S31508004EE002480068C0F30220704700000CED00E09D
S31508004EF010B5002804DB0A07130E054A135406E00A
S31508004F000A07140E034A00F00F031B1FD45410BDE2
S31508004F1000E400E018ED00E000BF704770B58AB005
S31508004F2004460D4604B3208864281DDA208A0A211F
S31508004F30B0FBF1F609A8032100220592CDE9062166
S31508004F400890208AE169CDE90116CDE90302207AA5
S31508004F5000902346064A29466068FDF773FB2188B8
S31508004F60044840F8214000BF38460AB070BD00002A
S31508004F70595300089C1300202DE9F0418AB00446D5
S31508004F800D4616461F46DDF840801C481C49086039
S31508004F9008464760C0F80880C4600661456100217C
S31508004FA00176417681760121C17600210177417724
S31508004FB0FBF744FC18B101200AB0BDE8F0810020D7
S31508004FC0059006900120079000200090019002901D
S31508004FD003900490012008900E200990694608481D
S31508004FE0FBF79AFB08B10220E6E70548FBF73AFD0E
S31508004FF008B10320E0E70020DEE700000064004077
S31508005000F415002010B5044600204FF0E021086191
S315080050100420FCF703FB0148046010BD741000204F
S3150800502070B5034600224FF0E02675690D4E3668C6
S3150800503003FB06F44FF0E026B16910E04FF0E026D6
S31508005040B06988420BD0884202D20E1A324402E076
S315080050502E1A0E4432440146A24200D300E0EDE780
S3150800506000BF70BD7410002010B50220FFF7D8FFEE
S3150800507010BD000000B587B000BF00BF002001903A
S315080050801A48006840F00200184908600846006897
S3150800509000F00200019000BF00BF00BF00BF00BFC4
S315080050A0002001900846006840F0020008600846A3
S315080050B0006800F00200019000BF00BF00BF40205A
S315080050C002900120039004900320059002A9084845
S315080050D0FBF760FD802002901120039002A9044886
S315080050E0FBF758FD00F006F807B000BD303802405F
S315080050F00004024010B500BF002280210C48FBF7CF
S315080051004BFE00BFFFF7B0FF00BF01224021084851
S31508005110FBF742FE00BFFFF7A7FF00BF0122802171
S315080051200348FBF739FE00BFFFF79EFF10BD0000DE
S315080051300004024070B506460C460025304600F0CD
S315080051401DF80546A54203D2601B00F005F802E0EB
S31508005150012000F001F870BD38B504466A46002102
S315080051602046FDF74DFD38BD02460020914201D389
S31508005170881A02E0C2F1FF335818704770B5044622
S3150800518000F008F8064631462046FFF7EDFF0546CB
S31508005190284670BD08B56846FDF790FD08BD0000B5
S315080051A038B5FBF789F800BFFFF7F4FF04460D4B47
S315080051B022460DA10020FFF74FF90EA10020FFF7A8
S315080051C04BF900BF6846FCF74DFE0EA11248FFF7E3
S315080051D0A5FE12A11648FFF7A1FE6846FDF74CF991
S315080051E0002038BDE653000825642025733E3E207E
S315080051F000000000424D53207374617274200D0A3A
S3150800520000000000706F6C6C5F73746172745F7479
S3150800521061736B3100000000140E0020706F6C6C17
S315080052205F73746172745F7461736B32000000009F
S315080052303C0E002000BFFEE738B5FBF7BFFD07238D
S31508005240022208214FF4A87000F018F8A820FFF7EA
S31508005250D9FEFCF7E3FB4FF4E1342046FCF79AFC51
S31508005260600506231A044FF4A00100900020FFF7FA
S3150800527083FEFFF7FFFE38BD00BFFEE72DE9F041CC
S3150800528092B080460C4615461E460027302106A8D1
S31508005290FBF71DF9142101A8FBF719F900BF002037
S315080052A000902A48006840F080502849086008465F
S315080052B0006800F08050009000BF00BF00BF0020CB
S315080052C000902348006840F4804021490860084659
S315080052D0006800F48040009000BF00BF01200690DF
S315080052E00004079002200C9041050D91CDF83C80F2
S315080052F00E941095119606A8FBF742FF07461FB1B4
S31508005300012012B0BDE8F0810F2001900220029022
S31508005310002003904FF4A05004904FF4805005905D
S31508005320052101A8FBF7ECFD07460FB10120E8E7C8
S31508005330FBF738FD41F20101884205D105480068AE
S3150800534040F48070034908600020DAE740380240DC
S3150800535000700040003C02402DE9F0410546002659
S31508005360002D26D02C46606908B16069804700BFC9
S3150800537000BFFFF70FFF07460F4B3A460FA1002065
S31508005380FFF76AF8FFF706FF871B22883B460EA140
S315080053900020FFF761F800BFFFF7FCFE0646002075
S315080053A0E0816089A169884761893046FFF7C2FEB6
S315080053B0DEE7BDE8F0810000EB53000825642025F0
S315080053C0733E3E20000000007461736B3A2564202A
S315080053D0706572696F643A25640D0A004FF0407073
S315080053E0E1EE100A70476D61696E007461736B5F58
S315080053F074656D706C617465006273705F74617357
S315080054006B5F626561745F77646F67000000000018
S315080054100000000001020304060708090000000056
S3150800542001020304303132333435363738394142D4
S3150800543043444546D81A00200600000040000000F4
S3150800544000010000D81B00208000000000020000B8
S315080054502000000000020000D81D00201E000000E9
S315080054600A000000D81F00200A000000640000009F
S315080054709001000040000000E80300001D00000045
S315080054800A000000682100200C00000080000000CF
S31508005490000200009008000001010000785634124E
S315080054A001010000000000000000000000000000EC
S315080054B000000000000000000000000000000000DE
S315080054C000000000000000000000000001010100CB
S315080054D02800040000000000000000000000000092
S315080054E000000000000000000000000000000000AE
S315080054F00000000001002000010010000C00100050
S31508005500000000000000000000000000000000008D
S31508005510000000000000000000000000000000007D
S31508005520000000000000000000000000000000006D
S3150800553001010100300001010C00200020000400D8
S315080055400400000000000000000000000000000049
S31508005550000000000000000000000000000000003D
S31508005560000000000000000000000000000000002D
S3150800557000000000010101013000010000000000E8
S31508005580000000000000000000000000000000000D
S3150800559000000000000000000000000000000000FD
S315080055A0000000000101010128000C008001000034
S315080055B0040101010101010100000101C400080004
S315080055C001010000000000000000000000000000CB
S315080055D000000000000000000000000000000000BD
S315080055E000000000000000000000000000000000AD
S315080055F0000000000101300050780000C1090000D9
S31508005600205600080000002038110000C4010008D8
S31508005610FC56000838110020C01A000020020008B5
S3150800562001FF01FF01FF01FF01FF01FF01FF01FF6C
S3150800563001FF01FF01FF01FF01FF01FF0122320106
S3150800564013400613200225F401D0071A90111339C6
S31508005650521B083504318220320213440D132005EB
S315080056606BE80328411A79288B040728A9581112D0
S315080056704C1A403A4A402B2B024044C1C20C1A48E5
S315080056802C3C0C0240392908D92DB92C3B1001585D
S31508005690492419080A19042C5D1802401090290497
S315080056A09A031829B5091218195D0913180A1280E0
S315080056B01829AC19800913180A150818199109131D
S315080056C01819910912782911F91829F809121829AF
S315080056D04829C171B91829C1E918196019BF0913F0
S315080056E01819BF0910189C0802405FB918995F99E4
S311080056F0A86119F339A81103B124F400CD
S7050800018968
